:02000000452891
:08000800042805140800A00003
:100010000930A100031003180514031C051020303B
:10002000A200A20B1128A00CA10B0B280514203054
:10003000A200A20B19280800A801A901AA01AB017E
:10004000AC01AD01AE01AF010408A5001830A3005A
:10005000A00DA10DA20D283084000830A400800D51
:10006000F630000703188000840AA40B2F28A30B86
:1000700028283030A807A907AA07AB07AC07AD07A7
:10008000AE07AF0725088400080083018B018A01B1
:100090008501073099008316A73081000C30850058
:1000A00083120520B101B201B301BA01BB013B08C3
:1000B000A0003A08A100A2011C202C0807202B0850
:1000C00007202A08072029080720280807202C30A5
:1000D00007203108A0003208A1003308A2001C202C
:1000E0002F0807202E0807202D0807202C0807209E
:1000F0002B0807202A08072029080720280807209E
:100100000D3007200A3007208519D5208B20BB0A27
:100110000319BA0A5728B001810100000000FB3022
:10012000B4001530B5001530B6008B0105308500E0
:1001300083160E30850083120B1DA128B00A0B1107
:10014000A428000000000000B40B9C28FB30B40081
:10015000B50B9C281530B500B60B9C280000D63096
:10016000B8000B1DB628B00A0B11B928000000001A
:100170000000B80BB1280530850083160C308500CF
:1001800083120108B2003008B300B901B90A85141E
:1001900085100B110108031132020319C628B90A90
:1001A000B909B90A390AB10008000930BB070318B8
:1001B000BA0A5130B4009F30B5001430B600B40B09
:0C01C000E228B50BE428B60BDF2808008D
:02400E00C13FB0
:00000001FF
